Subject: addendum to last message

From: Wu-chang Feng <[email-masked]>
Date: Wed, 16 Feb 2000 18:21:44 -0800

The situation gets worse when the connection is closed with
shutdown(fd,2).  Data segments continue to be sent to the Palm at the
exponential backoff interval.  (Note that shutdown maps to
NetLibSocketShutdown).  Am I looking at a NetLib bug?

Thanks in advance,
Wu

18:03:00.056635 166.137.17.102.9492 > mynetra.8005: . ack 1609 win 1876
18:03:00.056660 mynetra.8005 > 166.137.17.102.9492: . 2681:3217(536) ack 57 win 9112 (DF)
18:03:00.348836 166.137.17.102.9492 > mynetra.8005: . ack 2145 win 1876
18:03:00.348856 mynetra.8005 > 166.137.17.102.9492: . 3217:3753(536) ack 57 win 9112 (DF)
18:03:00.732199 166.137.17.102.9492 > mynetra.8005: . ack 2681 win 1876
18:03:00.732218 mynetra.8005 > 166.137.17.102.9492: . 3753:4289(536) ack 57 win 9112 (DF)
18:03:01.119171 166.137.17.102.9492 > mynetra.8005: . ack 3217 win 1876
18:03:01.119195 mynetra.8005 > 166.137.17.102.9492: . 4289:4825(536) ack 57 win 9112 (DF)
18:03:01.608295 166.137.17.102.9492 > mynetra.8005: F 57:57(0) ack 3753 win 1340
18:03:01.608314 mynetra.8005 > 166.137.17.102.9492: . ack 58 win 9112 (DF)
18:03:01.900139 166.137.17.102.9492 > mynetra.8005: F 57:57(0) ack 4289 win 0
18:03:01.900160 mynetra.8005 > 166.137.17.102.9492: . ack 58 win 9112 (DF)
18:03:02.381615 166.137.17.102.9492 > mynetra.8005: F 57:57(0) ack 4289 win 0
18:03:02.381651 mynetra.8005 > 166.137.17.102.9492: . ack 58 win 9112 (DF)
18:03:02.396155 166.137.17.102.9492 > mynetra.8005: F 57:57(0) ack 4289 win 0
18:03:02.396171 mynetra.8005 > 166.137.17.102.9492: . ack 58 win 9112 (DF)
18:03:02.480053 166.137.17.102.9492 > mynetra.8005: F 57:57(0) ack 4289 win 0
18:03:02.480070 mynetra.8005 > 166.137.17.102.9492: . ack 58 win 9112 (DF)
18:03:02.961498 166.137.17.102.9492 > mynetra.8005: F 57:57(0) ack 4289 win 0
18:03:02.961519 mynetra.8005 > 166.137.17.102.9492: . ack 58 win 9112 (DF)
18:03:02.976078 166.137.17.102.9492 > mynetra.8005: F 57:57(0) ack 4289 win 0
18:03:02.976096 mynetra.8005 > 166.137.17.102.9492: . ack 58 win 9112 (DF)
18:03:03.085505 166.137.17.102.9492 > mynetra.8005: F 57:57(0) ack 4289 win 0
18:03:03.085524 mynetra.8005 > 166.137.17.102.9492: . ack 58 win 9112 (DF)
18:03:03.446604 166.137.17.102.9492 > mynetra.8005: F 57:57(0) ack 4289 win 0
18:03:03.446624 mynetra.8005 > 166.137.17.102.9492: . ack 58 win 9112 (DF)
18:03:03.457563 166.137.17.102.9492 > mynetra.8005: F 57:57(0) ack 4289 win 0
18:03:03.457578 mynetra.8005 > 166.137.17.102.9492: . ack 58 win 9112 (DF)
18:03:03.639940 166.137.17.102.9492 > mynetra.8005: F 57:57(0) ack 4289 win 0
18:03:03.639958 mynetra.8005 > 166.137.17.102.9492: . ack 58 win 9112 (DF)
18:03:03.833246 166.137.17.102.9492 > mynetra.8005: F 57:57(0) ack 4289 win 0
18:03:03.833264 mynetra.8005 > 166.137.17.102.9492: . ack 58 win 9112 (DF)
18:03:03.946807 mynetra.8005 > 166.137.17.102.9492: . 4289:4825(536) ack 58 win 9112 (DF)
18:03:04.026944 166.137.17.102.9492 > mynetra.8005: F 57:57(0) ack 4289 win 0
18:03:04.026961 mynetra.8005 > 166.137.17.102.9492: . ack 58 win 9112 (DF)
18:03:04.220244 166.137.17.102.9492 > mynetra.8005: F 57:57(0) ack 4289 win 0
18:03:04.220263 mynetra.8005 > 166.137.17.102.9492: . ack 58 win 9112 (DF)
18:03:04.231195 166.137.17.102.9492 > mynetra.8005: F 57:57(0) ack 4289 win 0
18:03:04.231215 mynetra.8005 > 166.137.17.102.9492: . ack 58 win 9112 (DF)
18:03:04.439152 166.137.17.102.9492 > mynetra.8005: F 57:57(0) ack 4289 win 0
18:03:04.439174 mynetra.8005 > 166.137.17.102.9492: . ack 58 win 9112 (DF)
18:03:05.088229 166.137.17.102.9492 > mynetra.8005: . ack 4289 win 0
18:03:05.095516 166.137.17.102.9492 > mynetra.8005: . ack 4289 win 0
18:03:05.183051 166.137.17.102.9492 > mynetra.8005: . ack 4289 win 0
18:03:05.380049 166.137.17.102.9492 > mynetra.8005: . ack 4289 win 0
18:03:05.390995 166.137.17.102.9492 > mynetra.8005: . ack 4289 win 0
18:03:09.607223 mynetra.8005 > 166.137.17.102.9492: . 4289:4825(536) ack 58 win 9112 (DF)
18:03:10.885047 166.137.17.102.9492 > mynetra.8005: . ack 4289 win 0
18:03:20.938099 mynetra.8005 > 166.137.17.102.9492: . 4289:4825(536) ack 58 win 9112 (DF)
18:03:27.245048 166.137.17.102.9492 > mynetra.8005: . ack 4289 win 0
18:03:43.609735 mynetra.8005 > 166.137.17.102.9492: . 4289:4825(536) ack 58 win 9112 (DF)
18:03:44.723327 166.137.17.102.9492 > mynetra.8005: . ack 4289 win 0
18:04:28.952961 mynetra.8005 > 166.137.17.102.9492: . 4289:4825(536) ack 58 win 9112 (DF)
18:04:30.047417 166.137.17.102.9492 > mynetra.8005: . ack 4289 win 0
18:05:28.957296 mynetra.8005 > 166.137.17.102.9492: . 4289:4825(536) ack 58 win 9112 (DF)